:020000020000FC
:100000001FC01895189559C21895E2C202C11895DB
:100010001895189518951895189518951895189578
:06002000189518951895D3
:10004000F8944FED4DBF4EEF47BB48E341BB93984B
:10005000949895984EE041BD99279DBD9CBD42E086
:1000600049BF44E043BF40E040936B0040E0409311
:100070006D00BB27A0E740E35AE04D9343955A95A6
:100080005523D9F70E94FC0248B34F7048BB0E9429
:10009000950348B34F70406C48BB0E9495030E9483
:1000A000580348B34F70406248BB0E94950348B361
:1000B0004F70406A48BB0E9495030E94580348B3A2
:1000C0004F70406148BB0E94950348B34F70406633
:1000D00048BB0E9495030E94580378940E94EC0349
:1000E00010916B00109365001127109366000E9419
:1000F000160110916300103371F002E00E94CF03EB
:100100000E94B203109162000E94B203109161003C
:100110000E94B20315C010916200103351F002E04A
:100120000E94CF030E94B203109161000E94B203AB
:1001300007C01091610002E00E94CF030E94B20349
:1001400010916D00109365001127109366000E94B6
:10015000160110916300103371F002E40E94CF0386
:100160000E94B203109162000E94B20310916100DC
:100170000E94B20315C010916200103351F002E4E6
:100180000E94CF030E94B203109161000E94B2034B
:1001900007C01091610002E40E94CF030E94B203E5
:1001A0004FEF40936800409168004423E1F7977F48
:1001B0000E94E20090FDFECF98600E94E20090FD58
:1001C000FECFF5CF90FD089540916800442309F0DB
:1001D0000895F8941FB6916093FB16F0949A01C0AD
:1001E000959A0E9481030E9481034FEF48BF40E12E
:1001F0004093680044274DBD4CBD4AE849BF93FB7E
:1002000016F0949801C0959842E44EBD1FBE7894B4
:100210000895A8951FB62F9320916800222319F006
:100220002A95209368002F911FBE18951FB60F9333
:100230001F9388249924AA24BB240091650010915F
:100240006600202F312F085E134020F0B394202F3A
:10025000312FF9CF022F132F0456104020F0A39412
:10026000202F312FF9CF022F132F0A50104020F0EA
:100270009394202F312FF9CF022F132F802EBB27DD
:10028000A1E6FF27E0E7E80D00810D93E0E7E90D27
:1002900000810D93E0E7EA0D00810D93E0E7EB0D9F
:1002A00000810C931F910F911FBE08951FB60F93ED
:1002B0001F9393FB0EF001C05DC091FBEEF001E0D7
:1002C0000E94CF031DE30E94B203109164000E94BC
:1002D000B2031EE20E94B203109163000E94B203B7
:1002E000109162000E94B203109161000E94B2035B
:1002F00012E40E94B203DDC001E00E94CF0392FB32
:1003000026F41EE30E94B20303C01DE30E94B20361
:10031000109164001033C9F4109163000E94B2037D
:100320001EE20E94B203109162000E94B20310917B
:1003300061000E94B20312E40E94B20310E20E9424
:10034000B20310E20E94B203B4C00E94B203109143
:1003500063000E94B2031EE20E94B2031091620089
:100360000E94B203109161000E94B20312E40E9445
:10037000B2039FC001E40E94CF0394FB16F41EE376
:1003800001C01DE30E94B20340B340FB0EF401C064
:100390007AC041FB1EF442FB86F58BC010916400CD
:1003A0001033B1F4109163000E94B2031EE20E9468
:1003B000B203109162000E94B203109161000E948A
:1003C000B20311E40E94B20310E20E94B20371C0B2
:1003D0000E94B203109163000E94B2031EE20E94C9
:1003E000B203109162000E94B203109161000E945A
:1003F000B20311E40E94B2035CC010916400103398
:1004000069F5109163001033A9F4109162000E9405
:10041000B2031EE20E94B203109161000E94B20377
:1004200011E40E94B20310E20E94B20310E20E94A3
:10043000B2033FC00E94B203109162000E94B20357
:100440001EE20E94B203109161000E94B20311E407
:100450000E94B20310E20E94B2032BC00E94B203BA
:10046000109163000E94B203109162000E94B203D7
:100470001EE20E94B203109161000E94B20311E4D7
:100480000E94B20316C0109164000E94B2031EE2E3
:100490000E94B203109163000E94B20310916200A7
:1004A0000E94B203109161000E94B20311E40E9405
:1004B000B2031F910F911FBE08951FB644274EBD72
:1004C0004DBD4CBD42E049BF93FB1EF00E9495021A
:1004D00002C00E946D021FBE18951FB604B515B567
:1004E0002FE037E2201B310BA0F09F7E20916D00A2
:1004F000402F512F421B504018F0042F152F02C0DF
:100500000027112700936500109366008FDECEDE72
:1005100009C090610FE017E2009365001093660038
:1005200085DEC4DE9E7F1FBE08951FB604B515B5D7
:1005300091FBEEF02FE037E2201B310BA8F09B7F00
:1005400020916B00402F512F2F77421B504018F005
:10055000042F152F02C00027112700936500109368
:10056000660064DEA3DE31C0939A92602EC024ED53
:1005700033E0201B310B20F093989D7F9B7F25C09B
:100580002FE037E2201B310BB8F09B7F939A9260EB
:1005900020916B00402F512F2F77421B504018F0B5
:1005A000042F152F02C00027112700936500109318
:1005B00066003CDE7BDE09C094600FE017E200932A
:1005C00065001093660032DE71DE9E7F1FBE0895C7
:1005D0001FB60F9300270EBD0DBD0CBD0093650027
:1005E0000093660002E009BF21DE60DE9E7F0FEF10
:1005F00008BF0F911FBE1895C298C1980E94810331
:100600000E94810348B34F70406348BB0E9495032A
:100610000E94580348B34F70406348BB0E94950343
:100620000E94580348B34F70406348BB0E94950333
:100630000E94580348B34F70406248BB0E94950324
:100640000E94580348B34F70406248BB0E94950314
:1006500048B34F70406848BB0E9495030E945803FE
:1006600048B34F7048BB0E94950348B34F70406831
:1006700048BB0E9495030E94580348B34F7048BB83
:100680000E94950348B34F70406148BB0E94950398
:100690000E946D0348B34F7048BB0E94950348B356
:1006A0004F70406648BB0E9495030E94580308950E
:1006B0002FB64F9344E34A9500000000000000006D
:1006C000D1F74F912FBE08950000000000000000F8
:1006D000000000000000000008952FB64F935F93C4
:1006E00055E04FEF4A9500000000000000000000B8
:1006F00000000000B9F75A95A1F75F914F912FBE06
:1007000008952FB64F935F9352E44FEF4A95000040
:10071000000000000000000000000000B9F75A953A
:10072000A1F75F914F912FBE0895000000000000D7
:1007300000000000000000000000C39A000000005C
:1007400000000000000000000000000000000000A9
:10075000C39800000000000000000000000000003E
:10076000000008950FB64F935F93C29AC19858B393
:10077000412F407F5F70542B58BB0E94950358B3A4
:10078000412F4295407F5F70542B58BB0E949503C8
:100790000E945803C2985F914F910FBE08952FB6E3
:1007A0004F935F93C298C198006858B3402F407F21
:1007B0005F70542B58BB0E94950358B3402F42954D
:1007C000407F5F70542B58BB0E9495030E945803D2
:1007D0005F914F912FBE089500E00E94CF0315E571
:1007E0000E94B2031DE30E94B20300E40E94CF0303
:0E07F00019E40E94B2031DE30E94B2030895B3
:00000001FF
